:02000000B02F1F
:0A000600E808031D07280800F93080
:10001000FF3E031D0828E80B07280800FA30E80017
:100020000320FA30E8000320FA30E8000320FA3019
:10003000E8000320CF0B0E28080083120313861557
:10004000861108000230831203130605E90003102D
:10005000690CC5000800E908031930280615312885
:10006000061108006908EA0003106A0DE900023071
:100070006905E900FD300605EA0069086A048600A2
:100080000800630E0F3985001D20630885001D20C0
:100090000230E80003200800823083160313860034
:1000A00001308312E9002B2022204508E800E901F5
:1000B0002B200130E9003220803083168600831225
:1000C0006808C500080080308316031386000130DD
:1000D0008312E9002B20E9013220E9012B200800DE
:1000E00006106108013A03197A286108023A0319D7
:1000F0007F2889286208803EE30041208928E501A5
:100100006208403EE4000318E50A64088038E30012
:1001100041200230E80003200800780883169B0085
:100120001C141A088312C5000800FA01FC01FB0127
:100130006208FD006308FE00FA19AC28611CA628BD
:100140007D08FB070318FC0A7E08FC07E10C03107E
:10015000FD0DFE0DFA0A9C287B08C5007C08C60030
:100160000800FA01FC01FB016A08FD00FE01FA1912
:10017000C7286B1CC1287D08FB070318FC0A7E08F2
:10018000FC07EB0C0310FD0DFE0DFA0AB7287B08E7
:10019000C5007C08C6000800EE01ED01EC01EB0192
:1001A000EF016F1AEB280310EB0DEC0DE40DE50DDC
:1001B000ED0DEE0D67086E02031DE02866086D0266
:1001C000031CE9286608ED026708031CEE03EE0233
:1001D0006B14EF0AD1286D08C5006E08C600080030
:1001E00083120313E9012B20E90132200130E900D9
:1001F0002B200130E90032200800E2010830E30042
:10020000E4016408803A803C031D08296308003C2F
:10021000031822296208E8000310680DE20001308B
:1002200061056204E2006108E8000310680CE10067
:100230006408E500E3080319E5036303E3006508C8
:10024000E40001298030E300E4016408803A803C46
:10025000031D2C296308003C031846296208E900A5
:1002600032206208E8000310680CE2000130E90067
:100270002B20E9012B206308E6006408E700031047
:10028000E70C660CE3006708E40025294C20080011
:10029000ED01EC01EB01EA01EE016E1A6729031092
:1002A000EA0DEB0DE40DE50DEC0DED0D67086D02AB
:1002B000031D5C2966086C02031C65296608EC02B4
:1002C0006708031CED03ED026A14EE0A4D296A0863
:1002D000C5006B08C6000800E3016008303EA500B9
:1002E0000430E3006308003C0318CC2977297829FF
:1002F000DF1F8D295E09E4005F09E500E40F812915
:10030000E50A0A30E600E701CC204509E800460985
:10031000E900E80F8C29E90A99295E08E4005F08E2
:10032000E5000A30E600E701CC204508E800460871
:10033000E9006808303EEA00831320308400630837
:1003400084076A088000A429A529DF1FBA295E094D
:10035000E4005F09E500E40FAE29E50A0A30E60093
:10036000E70148214509E8004609E900E80FB929F5
:10037000E90AC6295E08E4005F08E5000A30E600E5
:10038000E70148214508E8004608E9006808DE0062
:100390006908DF00E30372295E08303EA000E30134
:1003A0006308053C031CED296308620783169B0064
:1003B00083128313203084006308840700088316A7
:1003C0009A001C1555309D00AA309D009C149C1865
:1003D000E7291C118312E30AD0290800DF015F0816
:1003E000053C031C002A5F085E07F8008D2083137C
:1003F000203084005F08840745088000DF0AEF2969
:10040000DF01250EF039F800F901F80CF80CF80CB2
:10041000780C0F39B0007908B100200EF039E000F7
:10042000600E0F39E1001030E2002730E300952024
:100430004508E7004608E800210EF039E400640EA4
:100440000F39E100E830E2000330E3009520450871
:10045000E5004608E60065086707EE006608EF005D
:1004600068080318EF0AEF07220EF039E900690E59
:100470000F39EA006430EB00B1204508EC00460873
:10048000ED006C086E07F3006D08F4006F080318A8
:10049000F40AF407230EF039F000700E0F39EA0069
:1004A0000A30EB00B1204508F1004608F20071085F
:1004B0007307F6007208F70074080318F70AF707C5
:1004C000240EF039F500750E0F397607F80077081D
:1004D000F9000318F90A7808C5007908C600080071
:1004E0005E08E1005F08E200702006146008E30087
:1004F00041200800DD015D08053C031CE02A570887
:10050000E1005D08053C5807E200702006145D0814
:10051000033A031D902A2E30E3004120DD0ADF2A32
:10052000912A922ADA1FA72A5909E4005A09E500FC
:10053000E40F9B2AE50A0A30E600E701CC204509D2
:10054000DE004609DF00DE0FA62ADF0AB32A5908BB
:10055000E4005A08E5000A30E600E701CC2045082F
:10056000DE004608DF005E08303EE3004120B82A86
:10057000B92ADA1FCE2A5909E4005A09E500E40F26
:10058000C22AE50A0A30E600E70148214509E200EF
:100590004609E300E20FCD2AE30ADA2A5908E4000B
:1005A0005A08E5000A30E600E70148214508E20064
:1005B0004608E3006208D9006308DA00DD0A7B2AF6
:1005C0005708E1005D085807E000DD0A6008E20016
:1005D000702006142C30E30041205708E1005D082C
:1005E0005807E000DD0A6008E20070200614F82ACF
:1005F000F92ADC1F0E2B5B09E4005C09E500E40F1F
:10060000022BE50A0A30E600E701CC204509DE00AE
:100610004609DF00DE0F0D2BDF0A1A2B5B08E40012
:100620005C08E5000A30E600E701CC204508DE0062
:100630004608DF005E08303EE3004120DD0108008F
:10064000C418272BDD01DE01DF01E001C414DC0149
:10065000DB0104305B025C080318302B0319322BDA
:10066000DC1F332B342B6A2B352B362BD81F472B13
:100670005709E4005809E500E40F3F2BE50A103064
:10068000E600E701CC204509E800E80A512B5708AD
:10069000E4005808E5001030E600E701CC204508EA
:1006A000E80083135D3084005B08840768088000DD
:1006B000570EE1000F30E105580EE200F039E10479
:1006C0000F30E2056108D7006208D800DB0F692B04
:1006D000DC0A292B63205A08E100FD205F0EF03967
:1006E000E200620E0F39E300600EF0396307E100AB
:1006F000FD205D0EF039E200620E0F39E3005E0E60
:10070000F0396307E100FD20CE30E100FD205908FB
:10071000E100FD20F020F03083168500F0308600E7
:10072000080083120313D10182308316860008303B
:100730008312D200D3015308803A803C031DA22BC0
:100740005208003C0318BC2B5108D5000310550D6E
:10075000D1000130E9002B20222045085104D100AE
:10076000E9012B205308D400D2080319D403520303
:10077000D2005408D3009B2B0130E90032205108ED
:10078000C500080083120313861106100530E80027
:100790000320033085001D200530E80003200230CF
:1007A00085001D200530E80003202830E3004120AB
:1007B0000530E80003200830E30041200530E80060
:1007C00003200C30E30041200530E8000320063010
:1007D000E30041200800D10151080F3C031C002C0C
:1007E0004F08E1005108E20070200614510850073C
:1007F000F8008D2037304502E3004120D10AEC2B70
:10080000D101080063204F08E100FD209123450835
:10081000D000F020F03083168500F030860083127F
:100820005008C50008008312031306100130E300CE
:1008300041200230E80003200800D201D10101303C
:10084000D300D401D601D5014208DE000B30DF0011
:100850007F30E00070221E30E800032032082E02B4
:10086000DB00330A031833082F02DC0038085B076B
:10087000DD003908DE005C080318DE0ADE075D08CB
:10088000DF005E08E0000310DF0DE00D0310DF0D58
:10089000E00D0310DF0DE00D30085F07E1003108C7
:1008A000E20060080318E20AE2076108D700620864
:1008B000D8004308D9004F08DA0020230130831202
:1008C000360603193708031D6A2C3208D100330895
:1008D000D2006E2C2E08D1002F08D2004208D7007B
:1008E0000330D8005108D9005208DA003008DB0084
:1008F0003108DC007A225108DE005208DF0030089F
:10090000E0003108E1005008E2006C212830E800E6
:100910000320D308031D8F2CD4080319AA2D060E1B
:100920000F390E3A031DA12C4208DE000B30DF0008
:100930002030E0007022B701B6010130D300D401AD
:100940000800060E0F39073A031D142D4208DE0079
:100950000230DF007E30E00070224208023A031DC0
:10096000C62CBE08031DBF2CBF08031DBF2CD830EA
:10097000AE000430AF000130BE00BF01C52CFC301A
:10098000AE000830AF00BF01BE01082DB608031D40
:10099000FF2CB708031DFF2CC008031DE32CC10862
:1009A000031DE32CF630AE002830AF007830DE00B7
:1009B000EE214508B2004608B300F030C300013014
:1009C000C000C101FF2C0130400603194108031D7E
:1009D000F52CFC30AE000830AF00B301B201F030AE
:1009E000C3000230C000C101FF2CD830AE0004307B
:1009F000AF00B301B2017030C300C101C0012E08C5
:100A0000DE002F08DF00E101E0015008E2006C2168
:100A1000C830E80003204208DE000230DF0020304A
:100A2000E0007022D401D30180300505D700DA013F
:100A3000003057020319DA0A060E0F39D800D9011F
:100A40000D3058020319D90A59085A04DD00060E60
:100A50000F39DB00DC010B305B020319DC0A5C0898
:100A60005D040319A92D40300505DE00E1010030C9
:100A70005E020319E10A060E0F39DF00E0010D30B6
:100A80005F020319E00A600861040319742DBA08B3
:100A9000031D4D2DBB080319652D013036060319C2
:100AA0003708031D572DB20F562DB30A642D3C088D
:100AB0002E07E2003D08E3002F080318E30AE307CE
:100AC0006208AE006308AF00732DB00F682DB10A45
:100AD0000A30300603193108031D732DAE0F712D36
:100AE000AF0AB101B001A72DBA08031D7A2DBB08CA
:100AF0000319922D0130360603193708031D852D81
:100B0000B2080319B303B203912D3C082E02E20090
:100B10003D0A03183D082F02E3006208AE00630897
:100B2000AF00A72DB0080319B103B0030030FF30A8
:100B30003106031DA72D3008FF3A031DA72DAE086F
:100B4000031DA32DAF03AE030930B000B101D401E2
:100B5000D301892C0130D300D40132082E02D700F2
:100B6000330A031833082F02D8005708D500580855
:100B7000D6000B305602031DBF2DB9305502031CA1
:100B8000DD2DD61BDD2DB208031DC92DB3080319B9
:100B9000D72D3208523ED7003308D800033003184F
:100BA000D80AD8075708AE005808AF00DB2D5230DE
:100BB000AE000330AF00B101B0015608033C031D85
:100BC000E32D5508513C0318E72DD61F012EB2081E
:100BD000031DED2DB3080319FB2D3208B83ED700D5
:100BE0003308D8000B300318D80AD8075708AE00CE
:100BF0005808AF00FF2DB830AE000B30AF00B10188
:100C0000B0012E2C83120313CA01C9010130CB009D
:100C1000CC010630CD00F03083168500F030860020
:100C20004030810083128B01C2236830DE00EE2148
:100C30004508A6004608A7003008A8003108A9000A
:100C40007030DE00EE214508AA004608AB003008EF
:100C5000AC003108AD007830DE00EE214508B2006E
:100C60004608B3000130CF004030D000EB23023003
:100C7000CF005030D000EB230230CF000E20CB0845
:100C8000031D452ECC0803196A2E0130CF00D00178
:100C9000EB230230CF001030D000EB230130D7001F
:100CA0000330D8002608D9002708DA002808DB001E
:100CB0002908DC007A220230D7000330D8002A0845
:100CC000D9002B08DA002C08DB002D08DC007A2282
:100CD000CC01CB0132082602D300330A03183308B3
:100CE0002702D40038085307D5003908D600540825
:100CF0000318D60AD6075508DB005608DC00031097
:100D0000DB0DDC0D0310DB0DDC0D0310DB0DDC0D4A
:100D100028085B07DD002908DE005C080318DE0AEE
:100D2000DE075D08D7005E08D8004308D900C6304A
:100D3000DA00202383122A08D3002B08D4000310E2
:100D4000D30DD40D0310D30DD40D0310D30DD40D3A
:100D50002C085307D5002D08D60054080318D60ACE
:100D6000D6075508D7005608D800F030D900C03053
:100D7000DA002023C7308312CF0002244508C800C0
:100D8000FF3A031DC62E3F30C700CD2E481FCB2E85
:100D90002A30C700CD2E2130C7000130DE000C30D4
:100DA000DF004708E0007022C130CF000224450870
:100DB000C800FF3A031DDF2E3F30C700EC2E481F4E
:100DC000E72E831605122A308312C700EC2E8316F5
:100DD000051621308312C7000230DE000C30DF0020
:100DE0004708E0007022060E0F39CE00073A0319BB
:100DF0000A2F4E080B3A03193F2F4E080C3A0319DD
:100E00006A2F4E080D3A0319922F4E080E3A031915
:100E1000AC2FAC2F13240130CF002030D000EB23B7
:100E2000BA08031D1F2FBB08031D1F2F0130BC0074
:100E3000BD010630CD000130BA00BB01312F0130B9
:100E40003A0603193B08031D2E2F0A30BC00BD01D2
:100E50000A30CD000230BA00BB01312FCD01BB01F9
:100E6000BA010130DE004D08DF002330E0007022BF
:100E70000130CF000E200130CB00CC01AC2F2A086E
:100E8000AE002B08AF002C08B0002D08B1000230D6
:100E9000C2003208C9003308CA00B301B201B90167
:100EA000B801C030CF007030D0001D242E08AA0039
:100EB0002F08AB003008AC003108AD004908B20083
:100EC0004A08B300E030B8000130B9000130CB006F
:100ED000CC01AC2F2708273C031D702F2608103C9F
:100EE0000318912FA71B912F13240130CF0030300E
:100EF000D000EB232608AE002708AF00B101B001F7
:100F00000130B600B7010130C2000130BA00BB01A8
:100F1000C630CF007830D0001D240130CB00CC018A
:100F20001324AC2F2608AE002708AF002808B00015
:100F30002908B1000130C200C630CF006830D000AF
:100F40001D242E08A6002F08A7003008A80031088D
:100F5000A9000130CB00CC013230E80003203F2E45
:100F6000831203134410C410F630A6002830A700E3
:100F7000A901A801A030AA000230AB00AD01AC016C
:100F8000AF01AE01B101B001B830B2002430B300FE
:100F9000B501B401B701B601E030B8000130B900C5
:100FA0000130BA00BB010130BC00BD010130BE0000
:100FB000BF010130C000C1010130C200F030C300E8
:060FC0008A110A12022E44
:0A4000000200020002000B000000A5
:02400E0050025E
:104200008900AF005700570057005700570057006C
:104210005700570057005700570084007F00B10037
:104220008B00AF005700570057005700570057004A
:104230005700570057005700570084007F00B10017
:104240005700670065006800840057005700680049
:104250008400570057006800670084007F00B100A9
:10426000860083005700570057005700570057003B
:104270005700570057005700570084007F00B100D7
:1042800080008E00690083007D007B00570078006D
:104290008B008D005700640089008B008F00640044
:1042A0008A008E00570089009C00A300650057001B
:1042B00069006500690065006900570067006C00CF
:1042C0002D002D002D002D002D002D002D002D0086
:1042D000310030003400380036003000FF00FF00AD
:1042E000300031003200340030003000FF00FF00A9
:1042F000300039003400300030003000FF00FF0093
:00000001FF
